:10333500754B061218D5203D04E53070F912191E9B
:10334500754B0612189580E822754B041218D5E5C1
:103355003070FC12191E754B041218957F0112135B
:103365000A7E007FFF8F051230B1DFF97E007FFFF7
:10337500900000C0071230F2EFF0A3D007DFF4226F
:10338500754B011218D5E53070C512191E754B0124
:1033950012189522754C0112130A7808303BFDE589
:0B33A5003E24301212DBC23BD8EA22AB
:100D52007584008550D28551D37584018552D28520
:100D620053D3E4F551F55030100685545085555152
:100D720030110CE5502556F550E5513557F55130F7
:100D82001210E5348535F0A42550F550E5F03551C3
:100D9200F551301310E50A8538F0A42550F550E5D9
:100DA200F03551F551301410E5118537F0A4255076
:100DB200F550E5F03551F551E4F553F55230181080
:100DC200855452855553E555C3953C4003853C53A4
:100DD200301916E557C3953B4003853C57E552252C
:100DE20056F552E5533557F553301A10E53485352B
:100DF200F0A42552F552E5F03553F553301B10E5BA
:100E02000A8538F0A42552F552E5F03553F55330F2
:100E12001C10E5118537F0A42552F552E5F0355343
:100E2200F553301D10E5188536F0A42552F552E52C
:100E3200F03553F553301E10E529853AF0A42552BA
:100E4200F552E5F03553F553301F10E52A8539F098
:100E5200A42552F552E5F03553F553E553C3953DBC
:100E62004003853D5322900ECF303F03120E8A304D
:070E72004003120E9A30420A
:100E790003120EBE304103120EBD304303120ECED3
:100E890022E50B2509F50BE50C3508F50C93F50A58
:100E990022E512250EF512E513350DF51393C3134B
:100EA900F8E5142510F514E515350FF51593C31359
:100EB90028F5112222E5192517F519E51A3516F530
:100EC9001A93F51822227F8285888C8F9295989B98
:100ED9009EA1A4A7AAADB0B3B6B9BBBEC1C3C6C9CA
:100EE900CBCED0D3D5D7D9DCDEE0E2E4E6E7E9EB37
:100EF900EDEEF0F1F2F4F5F6F7F8F9FAFBFCFCFD8A
:100F0900FDFEFEFEFEFEFEFEFEFEFEFDFDFCFCFB02
:100F1900FAFAF9F8F7F6F4F3F2F0EFEDECEAE8E7AC
:100F2900E5E3E1DFDDDBD8D6D4D1CFCDCAC8C5C270
:100F3900C0BDBAB7B4B2AFACA9A6A3A09D9A979405
:100F4900908D8A8784817E7A7774716E6B68656209
:100F59005F5C595653504D4A4744423F3C393734F8
:100F6900322F2D2A282624211F1D1B191816141269
:100F7900110F0E0C0B0A08070605040403020201EF
:100F8900010000000000000000000001010202034E
:100F99000405060708090A0B0D0E1011131516187A
:100FA9001A1C1E20222427292B2E303335383A3D8E
:100FB900404245484B4E515456595C606366696CD2
:060FC9006F7275787B7F5A
:10123800D2F4C2F5C2F675840F85F0C8121068742E
:101248000312128712105C740312128712103F12D5
:10125800103F740312128712103F74021212871281
:10126800103F74281212F374061212F3740E12123D
:10127800F374011212F312105C74801212F322C07C
:1012880000A2E092F3A2E192F2A2E292F1A2E3922A
:10129800F0D2F475840F85F0C8C2F47830D8FE8592
:1012A800F0C87830D8FED00022C00075840FA2E4C0
:1012B80092F3A2E592F2A2E692F1A2E792F0D2F4BA
:1012C80085F0C8C2F47830D8FE85F0C87830D8FEEA
:1012D800D00022EF75840FD2F5C2F685F0C812123D
:1012E800B112103F12128712103F2275840FC2F5F7
:1012F800C2F685F0C81212B112103F1212871210EE
:101308003F22EF14A2E492E6C2E4D2E71212F322DB
:10131800740F1212F322740D1212F3227F011213AA
:101328000A78107F201212DBD8F9227F1112130AD3
:1013380078107F201212DBD8F9227F0112130A7865
:10134800207F201212DBD8F922C0077F018004C059
:10135800077F1112130AD007C082C083C007EF7538
:10136800F0109013821210807810E493FF1212DBB1
:09137800A3D8F7D007D083D0827E
:10138100222020202020202020202020202020205A
:1013910020303132333435363738394142434445D0
:1013A10046202020525334323220544553542020B9
:1013B10020202020525332333220544553542020D0
:1013C1002020205445535420204641494C45442077
:1013D100202020544553542020504153534544204C
:1013E100202020454550524F4D2054455354202034
:1013F10020204155582052454C41592054455354C1
:101401002020205055534820544F2054414C4B200C
:101411002054455354203320434841522F535542C1
:101421002054455354204649584544205354524969
:101431004E54455354205641524942205354524927
:101441004E464143544F52592044454641554C5410
:101451002050524F4752414D4D494E47204D4F4428
:101461004553494D504C45582052455045415445EE
:10147100522020205245434F5244494E47202020BC
:01148100204A
:1030B100C2B6758400D2C2C2C6D2C6C2C4D2C5C20B
:1030C100C330C3FD74A0F5C2C2C5C2C330C3FD8EF7
:1030D100C2C2C330C3FD8FC2C2C330C3FD8DC2C2E1
:1030E100C330C3FDD2C4C2C320C4FD12105CD2B62A
:1030F10022758400C2C3D2C530C3FD74A0F5C2C21B
:10310100C5C2C330C3FD8EC2C2C330C3FD8FC2C2AC
:10311100C330C3FDC2C4D2C5C2C330C3FD74A1F55F
:10312100C2C2C5C2C330C3FDC2C2C2C330C3FD8562
:0A313100C207D2C4C2C320C4FD22AD
:0800030002148200000000005D
:08000B00021483000000000054
:080013000216060000000000C7
:08001B003200000000000000AB
:09002300320000000000000000A2
:08002B00021486000000000031
:08003300320000000000000093
:0A003B003200000000000000000089
:0900430032000000000000000082
:08004B0032000000000000007B
:08005300320000000000000073
:08005B000214E50000000000A2
:08006300320000000000000063
:08006B000214FD00000000007A
:0800730002148C0000000000E3
:08007B0002160700000000005E
:080083000214E200000000007D
:08008B0032000000000000003B
:100093000216250000000000000000000000000020
:1000A3003275FF0775FFDE75FFAD75840F75E107C8
:1000B30075E20475E34475840F75A43575A5097558
:1000C300A6FF75A7FF759CFF759D00759E00759F24
:1000D300F075D8FF75E8FF75F80F75AD0F758401DE
:1000E30075893075888F75840275893075888F7529
:1000F300840F758A80758C67780874FF0000000090
:100103000000000000000000D5E0F1D8EDE58C30E0
:10011300E7FB759701758A0043890475840075B7F9
:100123001075840F438901758D01758F01758E02DA
:100133007480D5E0FD438902E58930E4FB759702BD
:1001430075840075D10775840075BB0175BA007598
:10015300BCF075C70075C60075C5FF75C4FF75E8AB
:100163008175840275BB0475BA0075BCF175C60050
:1001730075C4FF75E88875840075D484758401752A
:10018300D484758400C2F8759A47759D1A43F8099B
:1001930075870075840075B90075A90075910075A0
:1001A300985075840175981075840075C04075C3A7
:1001B3000075CFC9758400758E0075892075880513
:1001C300758400758A00758B6F758CF4758D6F431C
:1001D300885075840075C90075CA0075CB0075CC4D
:1001E3000075CD0075C80075840175C91875CA807E
:1001F30075CBFB75CDFB75CC80D2CA75840275C9EE
:100203001875CA1275CBF775CDF775CC12D2CA75AE
:10021300840075EF0075A8AF75B80075E6A475E79F
:100223001775F60075F7019000007F007E20E4F05B
:03023300A3DFFC4A
:10023600DEFA7808760008B880FA7535FF7536FF5D
:100246007537FF7538FF7539FF753AFF753BFF75D2
:100256003CFF753DFF752200752300751F0675204E
:080266000A751E0A755B0022F7
:1014820032C28D32758400C2CF32C0E0C083C082C6
:10149200C0D0C000C0F0C2CFB245204523120D52C9
:1014A200151BE51B7009751B0A7584017588AF153C
:1014B2001CE51C7009751C607584027588AF800E6E
:1014C200120E68152BE52B7005752B04D28B7584D3
:1014D20000D2ECD0F0D000D0D0D082D083D0E03295
:1014E200C2CF32C0E0C0D0E52C6002152CE52F60DF
:1014F20002152F75888FD0D0D0E032C0E0C0D0C0A6
:1015020084203C1375840F30DF25E5E8540FF53E47
:10151200D23C753FC88018153FE53F7006E53ED2C4
:10152200E7F53E75840F20DF06C23CD23BD2312064
:101532003E1475840F30F826E5E854F0C4F540D225
:101542003E7541C880181541E5417006E540D2E775
:10155200F54075840F20F806C23ED23DD230E52D0B
:101562006002152DE55A6002155AE55C6002155CB1
:10157200E56960021569151DE51D707F751D0AE597
:101582002E6002152EE53060021530E56560021509
:1015920065E54D6002154DE54E6002154EE54F6062
:1015A20002154FE55D6002155DE55F6002155FE5BE
:0D15B2005E6002155EE56060021560151EAA
:1015BF00E51E703A751E0A12167CE5686002156802
:1015CF00E56360021563151FE51F7022751F06B2D4
:1015DF00A0E566600215661520E520701175200ADA
:1015EF00B2A1E56160021561E56260021562D08407
:1015FF00C28DD0D0D0E03232203A0DD23A85BF57CB
:10160F0085BE5675BB01800BC23A85BF5585BE544A
:10161F0075BB00C2ED32C0E0C0D0E542B4000A0590
:10162F004285BE3475BB07803DB4010A054285BEB5
:10163F003175BB048030B4020A054285BE3475BBD8
:10164F00068023B4030A054285BE3275BB0480169B
:10165F00B4040A054285BE3475BB05800975420086
:10166F0085BE3375BB04C2EDD0D0D0E032E55B60F0
:04167F0002155B22D3
:100FCF0075840FD2FD2275840FC2FD2275840FD256
:100FDF00FC2275840FC2FC2275840FD2FED224220C
:100FEF0075840FC224C2FE22C29322D2932275842B
:100FFF000FA2FA2275840FA2F92275840FA2DD22A7
:10100F0075840FA2DE22A2922275840FA2DA2275B6
:10101F00840FA2DB2275840FA2D82275840FA2D968
:10102F00220000000000000000000000000000226D
:10103F00C000C001790478B4D8FED9FAD001D0002D
:10104F0022C000781412103FD8FBD00022C0E075E8
:10105F002C05E52C70FCD0E022C0E0752C0FE52CA0
:10106F0070FCD0E022C0E0752C64E52C70FCD0E061
:10107F0022A42582F582E58335F0F58322B40A0098
:10108F0022C0E0C3997001D3D0E022B506012250EF
:10109F0007B5070122400122D322EF75F0648424A3
:1010AF0030900061F0E5F0A375F00A842430F0A3CE
:1010BF00E5F02430F022EF75F06484243090006165
:0710CF00F0E5F0A375F00A43
:1010D600842430F0A3E5F02430F0900061E0B430D1
:1010E6000B7420F0A3E0B430037420F02290000EBD
:1010F600E0540FFFA3E0B420028019540FCF75F01F
:101106000AA42FFFA3E0B420028009540FCF75F084
:101116000AA42FFF22C006C005C00490000EE054AA
:101126000FFFFEA3E0B42003C3802C540FFDCF7540
:10113600F00AA42FFFA3E0B42003C3801A540FFCC7
:10114600EE75F064A420D20EFEED75F00AA42E40D2
:10115600052C40028001D3D004D005D0062275F0BC
:101166006484F6E5F00875F00A84F608A6F008220D
:10117600C0017900E6B4FF028027F908E6B4FF0350
:10118600C38022E975F00AA426F908E6B4FF03C372
:101196008013E975F00AA420D207C3264003F9801C
:1011A60004D3D00122E9D00122E675F00AA408266C
:1011B600227845EE12116475430075440078479015
:0411C6001210790882
:1011CA00EF134007A3A3A3A3A3801CC0E0C000C0E1
:1011DA0001C37905E49336D4A2E4540FF6A318D9CF
:1011EA00F3D001D000D0E0D9D8E543600C754409AA
:1011FA0075450975460975470985444385454485FA
:10120A004645854746220605020000020105000000
:10121A00040200010008040002000609000400029A
:0E122A00090108000408030601080607020374
:10026E0044313233343536373839302A234142431C
:10027E0044AAA3C1C2C3C4D7ABA8A92A23414243EF
:10028E000101010101010101010000000000000057
:10029E000000000000000000000000000000000050
:1002AE000000000000000000000000000000000040
:1002BE000000000000000000000000000000000030
:1002CE000000000000000000000000000000000020
:1002DE00000000000000000000000101010101010A
:1002EE0001010100000000000000000000000000FD
:1002FE0000000000000000000000000000000000F0
:10030E0000000000000000000000000000000000DF
:10031E0000000000000000000000000000000000CF
:10032E0000000000000000000000000000000000BF
:10033E0000000000010101010101010101000000A6
:10034E00000000000000000000000000000000009F
:10035E00000000000000000000000000000000008F
:10036E00000000000000000000000000000000007F
:10037E00000000000000000000000000000000006F
:10038E00000000000000000000000000000001015D
:10039E000101010101010100000000000000000048
:1003AE00000000000000000000000000000000003F
:1003BE00000000000000000000000000000000002F
:1003CE00000000000000000000000000000000001F
:1003DE00000000000000000000000000000000000F
:1003EE0000000000000000000101010101010101F7
:1003FE0001000000000000000000000000000000EE
:10040E0000000000000000000000000000000000DE
:10041E0000000000000000000000000000000000CE
:10042E0000000000000000000000000000000000BE
:10043E0000000000000000000000000000000000AE
:10044E000000010101010101010101000000000095
:10045E00000000000000000000000000000000008E
:10046E00000000000000000000000000000000007E
:10047E00000000000000000000000000000000006E
:10048E00000000000000000000000000000000005E
:10049E0000000000000000000000000020202020CE
:1004AE00202020202020202020202020202020203E
:1004BE00202020202020202020202020202020202E
:1004CE00202020202020202020202020202020201E
:1004DE00202020202020202020202020202020200E
:1004EE0020202020202020202020202020202020FE
:1004FE0020202020202020202020202020202020EE
:10050E0020202020202020202020202020202020DD
:10051E0020202020202020202020202020202020CD
:10052E0020202020202020202020202020202020BD
:10053E0020202020202020202020202020202020AD
:10054E00202020202020202020202020202020209D
:10055E00202020202020202020202020202020208D
:10056E00474C4F42414C2020202020202043544312
:10057E00535320434F444520202020202020444325
:10058E005320434F44452020202020204C545220FD
:10059E005245504541544552202020205350454548
:1005AE0044204449414C494E472020205350454554
:1005BE00442043414C4C494E472020202050544368
:1005CE00204E554D424552202020202020564F4986
:1005DE004345204D455353414745532020564F49DF
:1005EE00434520504C41594241434B202020494E17
:1005FE0056414C49442054595045202020204F55F7
:10060E0054204F462052414E4745202020494C4C05
:10061E004547414C2056414C554520204D5553548D
:10062E002046494C4C204649454C44202020494CFC
:10063E004C4547414C20434F4445202020444154D3
:10064E004120414343455054454420204C494E459A
:10065E00204E554D4245523A2020202055534552AA
:10066E002050524F4752414D4D494E4755534552DA
:10067E002049443A2020202020202020564F494354
:10068E0045205245434F5244494E472020494C4C39
:10069E004547414C20454E545259202020494C4C40
:1006AE004547414C2047414E4720202020202043E3
:1006BE004F4D504C45544544202020203633303683
:1006CE0037303639343731393734343737303739C4
:1006DE0037383235383534383835393135393438AC
:1006EE0039373431303031303331303731313031D8
:1006FE0031343131383132333132373133313133C4
:10070E0036313431313436313531313536313539A2
:10071E003136323136353136373137313137333193
:10072E003737313739313833313836313839313965
:10073E003231393631393932303332303632313076
:10074E003231383232353232393233333234313269
:10075E003530323534303036303037303135303167
:10076E003730323130323330323530323630333159
:10077E003033323033363034333034373035303046
:10078E00353130353330353430363530373130372A
:10079E00323037333037343131343131353131361F
:1007AE00313232313235313331313332313334311A
:1007BE0034313134333134353135323135353135FB
:1007CE0036313632313635313732313734323035E3
:1007DE0032313232313432323332323532323632E3
:1007EE0034333234343234353234363235313235C4
:1007FE0032323535323631323633323635323636AE
:10080E0032373132373433303633313133313533A9
:10081E003235333331333332333433333436333595
:10082E00313335363336343336353337313431317F
:10083E00343132343133343233343331343332347D
:10084E003435343436343532343534343535343653
:10085E003234363434363534363635303335303648
:10086E003531363532333532363533323534363539
:10087E003635363036363132363234363237363326
:10088E003136333236353436363236363437303317
:10089E003731323732333733313733323733343708
:1008AE0034333735344142434445464748494A4B31
:1008BE004C4D4E4F505152535455565758595A61EC
:1008CE0062636465666768696A6B6C6D6E6F707182
:1008DE0072737475767778797A303132333435367F
:1008EE00373839607E21402324255E262A28295F49
:1008FE002D2B3D7B7D5B5D7C3A3B3C3E2C2E3F2F72
:10090E002020202020202020206401001102251507
:10091E000101640200110325150101640400110494
:10092E002515010164080011052515010178060140
:10093E001106011901018201071107261501028214
:10094E00010811080115010782010911090115019C
:10095E000782010A110A0115010782010B110B0111
:10096E0015010782010C110C2715010982010D11C9
:10097E000D2715010982010E110E2715000982019E
:10098E000F110F271500098202101110281501638F
:10099E0082021111112915016382021211122A15F8
:1009AE00006382021311132A1500638202141114BC
:1009BE002B15006382031511152C1500FF820316EB
:1009CE0011162C1500FF82011711172F1500048226
:1009DE00011811182F15000482031911192C150A6C
:1009EE00FF82031A111A2C1500FF82031B111B2CF8
:1009FE001500FF82021C111C2B15016382021D11B2
:100A0E001D2B150163641000111E2D1501018203AB
:100A1E001E111F2C1500FF82021F11202B150163C2
:100A2E0082022011212B15016364200011222D1545
:100A3E00000182032111232C1500FF6440001124B4
:100A4E002E150001202020202020202020202020D4
:100A5E002020202020202020202020202020202088
:100A6E00202020202054454C434F2050524F4752B7
:100A7E00414D202020524144494F2050524F475261
:100A8E00414D20202050484F4E452050524F475246
:100A9E00414D202020434F4D50552050524F47522C
:100AAE00414D2020202041434345535320434F4482
:100ABE00452020204E554D4245525F4F465F494ED0
:100ACE005055545353454E53455F414C41524D5F23
:100ADE004D53472020434F535F414C41524D5F4D84
:100AEE005347202053454E53455F524553544F5262
:100AFE005F4D5347434F535F524553544F52455FDB
:100B0E004D53472053454E53455F414C4D5F524523
:100B1E005045415420434F535F414C4D5F52455019
:100B2E004541542053454E53455F5253545F5245F1
:100B3E005045415420434F535F5253545F524550DA
:100B4E00454154204D53475F5245504541545F49EE
:100B5E004E544552494E544552414C41524D5F49B7
:100B6E004E544552205455524E5F4F4E5F44454CA5
:100B7E0041592020205455524E5F4F46465F444502
:100B8E004C4159205455524E5F41524F554E445F81
:100B9E00444C592044544D465F54454C434F5F4C92
:100BAE004556454C44544D465F524144494F5F4C67
:100BBE004556454C564F49435F505245414D505F47
:100BCE004741494E2052585F505245414D505F4764
:100BDE0041494E20564F49435F54524E534D49544E
:100BEE005F4C564C424545505F524144494F5F4C15
:100BFE004556454C424545505F54454C434F5F4C1E
:100C0E004556454C53454E53455F41435155495FFB
:100C1E0054494D4553454E53455F52454C45415FF2
:100C2E0054494D452053454E53455F504F4C41520C
:100C3E004954592053454E53455F545249475F56C8
:100C4E004F4C542020434F535F414351555F5449FD
:100C5E004D452020434F535F52454C454153455F10
:100C6E0054494D452020434F535F504F4C415249FC
:100C7E0054592020434F535F545249474745525FC2
:100C8E00564F4C542020425553595F4C4F434B4FB7
:100C9E0055542020202020202020202020202020DD
:100CAE00313D454E202020202020202020202020B5
:100CBE004E4D425220202020202020202020205443
:100CCE00494D455320202020202020202020202068
:100CDE00204D494E20202020202020202020202082
:100CEE00205345432020202020202020202020316A
:100CFE0030204D5320202020202020202020313055
:100D0E0030204D5320202020202020202020205233
:100D1E004154494F20202020202020202020203107
:100D2E003D504F5320202020202020313D4C4F435A
:100D3E004B4F5554202020202020202020202053AF
:040D4E0043414C458C
:10454600756664E4900000F030260B302524124195
:10455600B112168380F530270B3025161241F01262
:10456600168380F530280B302508121A141216838C
:0345760080F522AB
:10168300E5667012900000E0D394004009C226C2C0
:1016930027C228C22522900000E0122C76179A0058
:1016A300179D0117A00217A30317A60417A8051770
:1016B300AA0617AC0717AF0817B20A17B50B17B866
:1016C3000F17BB1017BE1417C11517C41917C71A64
:1016D30017CA1B17CD1E17D01F17D32317D62417CE
:1016E300D92817DC2917DF2D17E22E17E52F17E866
:1016F3003017EB3217EE3317F03417F33517F66460
:1017030017F96517FC6617FF6718026E18046F1840
:101713000670184871180878180A79180C7A18484E
:101723007B180E8218108318128418148518178CCE
:10173300181A8D181C8E181E8F18219618249718A6
:101743002698182899182BA0182EA11831A21833FF
:10175300A31836AA1838AB183BAC183DAD1840B4E3
:101763001843B51846B61848B7184ABE184DBF18DF
:1017730050C01853C11848C21859F0185CF1185FCB
:10178300F21862FA1865FB1868FC186BFD186EFEF8
:101793001871FF00001874024C6B024AB80240B281
:1017A30002499D800480028000023F52021B820294
:1017B3004610021FA7023C850220F5023CDA0222F2
:1017C30043024133023A6702277B023E1F02239101
:1017D300023E6C0224DF023EB902262D0247950227
:1017E3004391023FE5123F9C023B2380000236688F
:1017F30002406F023D2F02402B024471023B7D8069
:10180300468032804B80408022804580078026803E
:101813003F023F06022C9C801C8035023D80023132
:10182300C08008802B024172022E1C0235F98020F1
:10183300022D5C80120233B08016021E4E02323D2E
:10184300023743800B800C023429023DD00230144E
:1018530002422F023C2F0249C40237AC024C8902D8
:101863003BD7024D11024D12024D130236D6024DE3
:0718730014E4900000F022D4
:0F4C6B00E4900002F0756664900000E004F0220F
:104AB8001213241213337BFF7A06796A1246477F52
:0F4AC8001112130AC22CC229900000E004F02240
:1040B20030293D900001E0FFC229BF2A079000008D
:1040C200E004F022EF642370277F231212DB9000BA
:1040D20002E004F0E0C394034010C226C227C228C3
:1040E200C225E4900000F00243CA9000007402F07E
:0140F20022AB
:10499D007BFF7A06796A1246471213337F11121381
:1049AD000A124C97E490003DF07F2A1212DBC22CC4
:0749BD00900000E004F0226D
:103F5200302946900001E0F56BC229E56B642A60C6
:103F620038AF6B124C7A5022AF6B1212DB90003DCD
:103F7200E02404F582E43400F583E56BF090003D23
:103F8200E004F0900000E004F0227BFF7A06799AC8
:093F920012464790000074FAF099
:013F9B002203
:101B8200202903021CEC900001E0FFC229BF2A07B2
:101B92009000007403F022EF64236003021CDD1244
:101BA20012DB900005E064397077A3E0643970714C
:101BB200A3E06439706BD22E900004E0FFB43108C8
:101BC200E4900037F0021C4CEFB43208E490003885
:101BD200F0021C5FEFB43302803E900004E0FFB4D9
:101BE2003408E4900039F0021C8DEFB43508E4901B
:101BF200003AF0021CA3EFB43608E490003BF00276
:101C02001CB9EFB437028010900004E0B4380280AF
:101C120007900004E0B4390B7BFF7A0679AA021C14
:101C2200E3C22E900004E0FFB43016A3E0B43011FA
:101C3200A3E0B4300CA3E0B43007900000740AF0C3
:101C420022EFB4310C123AC65007900000740FF024
:101C520022900004E0B4320C1239A7500790000021
:101C62007414F022900004E0B43311A3E0B4300CF9
:101C7200124A5750079000007419F022900004E0B5
:101C8200B4340FA3E0B4300A124BF3900000741E78
:101C9200F022900004E0B4350FA3E0B4300A124CF5
:101CA200089000007423F022900004E0B4360FA3E1
:101CB200E0B4300A124C1D9000007428F02290000B
:101CC20004E0B43716A3E0B43011A3E0B4300CA39F
:101CD200E0B43007900000742DF0227BFF7A067981
:0A1CE2009A12464790000074FAF0D1
:011CEC0022D5
:1046100090003C740BF090003D7407F0E490004E65
:10462000F090004FF0900050F07BFF7A05796A120D
:1046300046471246727F1E12130A9000007432F031
:014640002257
:101FA70012349ED3900067E09423900066E094007B
:101FB700400A12464190000074FAF022900066E051
:101FC700FEA3E0FF90091775F009122C6AEE75F071
:101FD70009A42583F583E493900045F090091875CB
:101FE700F009EF122C6AEE75F009A42583F583E456
:101FF70093900046F0900066A3E090091975F009E8
:10200700122C6AEE75F009A42583F583E4939000FA
:1020170047F090091A75F009EF122C6AEE75F0096E
:10202700A42583F583E493900048F0900066A3E02D
:1020370090091B75F009122C6AEE75F009A4258327
:10204700F583E493FD900049F090091C75F009EFC2
:10205700122C6AEE75F009A42583F583E4939000AA
:102067004AF0900066A3E090091D75F009122C6AEA
:10207700EE75F009A42583F583E49390004BF09067
:10208700091E75F009EF122C6AEE75F009A4258375
:10209700F583E49390004CF0900066A3E090091F4D
:1020A70075F009122C6AEE75F009A42583F583E40F
:1020B7009390004DF0ED6015900049E075F010A485
:1020C7002452F9740A35F0FA7BFF12464790004A0A
:1020D700E0FF601175F010A42452F9740A35F0FA84
:0E20E7007BFF124678900045E0900000F0224A
:103C850090003C7410F090003D7407F090004E7465
:103C950064F090004F740AF0900037E0900050F007
:103CA5007BFF7A05797A1246471246727F0D121309
:103CB5000A900005E0FF1212DB900006E0FF1212E9
:103CC500DB900007E0FF1212DB7F1E12130A900043
:053CD500007432F02232
:1020F50012349ED3900067E09400900066E094004F
:10210500400A12464190000074FAF022900066E001
:10211500FEA3E0FF90028E75F009122C6AEE75F0B1
:1021250009A42583F583E493900045F090028F750B
:10213500F009EF122C6AEE75F009A42583F583E406
:1021450093900046F0900066A3E090029075F00928
:10215500122C6AEE75F009A42583F583E4939000AB
:1021650047F090029175F009EF122C6AEE75F009AF
:10217500A42583F583E493900048F0900066A3E0DE
:1021850090029275F009122C6AEE75F009A4258368
:10219500F583E493FD900049F090029375F009EF03
:1021A500122C6AEE75F009A42583F583E49390005B
:1021B5004AF0900066A3E090029475F009122C6A2B
:1021C500EE75F009A42583F583E49390004BF09018
:1021D500029575F009EF122C6AEE75F009A42583B6
:1021E500F583E49390004CF0900066A3E09002968E
:1021F50075F009122C6AEE75F009A42583F583E4C0
:102205009390004DF0ED6015900049E075F010A435
:1022150024AAF9740435F0FA7BFF12464790004A68
:10222500E0FF601175F010A424AAF9740435F0FAE2
:0E2235007BFF124678900045E0900000F022FA
:103CDA0090003C7415F090003D7407F090004E740B
:103CEA00C8F090004F740AF0900038E0900050F04D
:103CFA007BFF7A05798A1246471246727F0C1213A5
:103D0A000A900005E0FF1212DB900006E0FF121293
:103D1A00DB900007E0FF1212DB7F1E12130A9000ED
:053D2A00007432F022DC
:1022430012349ED3900067E09400900066E09400FF
:10225300400A12464190000074FAF022900066E0B2
:10226300FEA3E0FF9002E875F009122C6AEE75F008
:1022730009A42583F583E493900045F09002E97562
:10228300F009EF122C6AEE75F009A42583F583E4B7
:1022930093900046F0900066A3E09002EA75F0097F
:1022A300122C6AEE75F009A42583F583E49390005C
:1022B30047F09002EB75F009EF122C6AEE75F00906
:1022C300A42583F583E493900048F0900066A3E08F
:1022D3009002EC75F009122C6AEE75F009A42583BF
:1022E300F583E493FD900049F09002ED75F009EF5A
:1022F300122C6AEE75F009A42583F583E49390000C
:102303004AF0900066A3E09002EE75F009122C6A81
:10231300EE75F009A42583F583E49390004BF090C8
:1023230002EF75F009EF122C6AEE75F009A425830C
:10233300F583E49390004CF0900066A3E09002F0E4
:1023430075F009122C6AEE75F009A42583F583E470
:102353009390004DF0ED6015900049E075F010A4E6
:1023630024CAF9740435F0FA7BFF12464790004AF9
:10237300E0FF601175F010A424CAF9740435F0FA73
:0E2383007BFF124678900045E0900000F022AB
:104133007BFF7A05799A1246477BFF7A06797A12D2
:1041430046787F0E12130A900006E0FF1212DB90EE
:104153000007E0FF1212DB7F1A12130A90003C746F
:0F4163001AF090003D7404F09000007432F022C6
:103A6700302F079000007403F0221246727F1E1257
:103A7700130A123814900068E0FEA3E0FFD3940005
:103A8700EE94004030EF94FBEE9400502890003CF9
:103A9700741BF090003D7407F090004E742CF0906A
:103AA700004F740AF0900036E014900050F0900038
:0F3AB700007432F02212464190000074FAF0229F
:10277B00D3900067E09400900066E09400400A124A
:10278B00464190000074FAF022900066E0FEA3E050
:10279B00FF90034275F009122C6AEE75F009A4251F
:1027AB0083F583E493900045F090034375F009EFB4
:1027BB00122C6AEE75F009A42583F583E49390003F
:1027CB0046F0900066A3E090034475F009122C6A62
:1027DB00EE75F009A42583F583E493900047F09000
:1027EB00034575F009EF122C6AEE75F009A42583E9
:1027FB00F583E493900048F0900066A3E0900346C5
:10280B0075F009122C6AEE75F009A42583F583E4A3
:10281B0093FD900049F090034775F009EF122C6A75
:10282B00EE75F009A42583F583E49390004AF090AC
:10283B000066A3E090034875F009122C6AEE75F060
:10284B0009A42583F583E49390004BF0900349751D
:10285B00F009EF122C6AEE75F009A42583F583E4D9
:10286B009390004CF0900066A3E090034A75F0093A
:10287B00122C6AEE75F009A42583F583E49390007E
:10288B004DF0ED6015900049E075F010A424EAF9C5
:10289B00740435F0FA7BFF12464790004AE0FF6064
:1028AB001175F010A424EAF9740435F0FA7BFF12C9
:0B28BB004678900045E0900000F022FD
:103E1F0090003C741FF090003D7407F090004E74BA
:103E2F0090F090004F740AF0900039E0900050F03D
:103E3F007BFF7A0579AA1246471246727F0F12133B
:103E4F000A900006E0FF1212DB900007E0FF12124B
:0D3E5F00DB7F1E12130A9000007432F02267
:1023910012349ED3900067E09400900066E09400B0
:1023A100400A12464190000074FAF022900066E063
:1023B100FEA3E0FF90039C75F009122C6AEE75F004
:1023C10009A42583F583E493900045F090039D755E
:1023D100F009EF122C6AEE75F009A42583F583E468
:1023E10093900046F0900066A3E090039E75F0097B
:1023F100122C6AEE75F009A42583F583E49390000D
:1024010047F090039F75F009EF122C6AEE75F00901
:10241100A42583F583E493900048F0900066A3E03F
:102421009003A075F009122C6AEE75F009A42583BA
:10243100F583E493FD900049F09003A175F009EF55
:10244100122C6AEE75F009A42583F583E4939000BC
:102451004AF0900066A3E09003A275F009122C6A7D
:10246100EE75F009A42583F583E49390004BF09079
:1024710003A375F009EF122C6AEE75F009A4258308
:10248100F583E49390004CF0900066A3E09003A4E0
:1024910075F009122C6AEE75F009A42583F583E421
:1024A1009390004DF0ED6015900049E075F010A497
:1024B100240AF9740535F0FA7BFF12464790004A69
:1024C100E0FF601175F010A4240AF9740535F0FAE3
:0E24D1007BFF124678900045E0900000F0225C
:103E6C0090003C7424F090003D7407F090004E7468
:103E7C00F4F090004F740AF090003AE0900050F08B
:103E8C007BFF7A0579BA1246471246727F0F1213DE
:103E9C000A900006E0FF1212DB900007E0FF1212FE
:0D3EAC00DB7F1E12130A9000007432F0221A
:1024DF0012349ED3900067E09400900066E0940061
:1024EF00400A12464190000074FAF022900066E014
:1024FF00FEA3E0FF9003F675F009122C6AEE75F05B
:10250F0009A42583F583E493900045F09003F775B4
:10251F00F009EF122C6AEE75F009A42583F583E418
:10252F0093900046F0900066A3E09003F875F009D1
:10253F00122C6AEE75F009A42583F583E4939000BD
:10254F0047F09003F975F009EF122C6AEE75F00958
:10255F00A42583F583E493900048F0900066A3E0F0
:10256F009003FA75F009122C6AEE75F009A4258311
:10257F00F583E493FD900049F09003FB75F009EFAC
:10258F00122C6AEE75F009A42583F583E49390006D
:10259F004AF0900066A3E09003FC75F009122C6AD4
:1025AF00EE75F009A42583F583E49390004BF0902A
:1025BF0003FD75F009EF122C6AEE75F009A425835F
:1025CF00F583E49390004CF0900066A3E09003FE37
:1025DF0075F009122C6AEE75F009A42583F583E4D2
:1025EF009390004DF0ED6015900049E075F010A448
:1025FF00242AF9740535F0FA7BFF12464790004AFA
:10260F00E0FF601175F010A4242AF9740535F0FA73
:0E261F007BFF124678900045E0900000F0220C
:103EB90090003C7429F090003D7407F090004E7416
:103EC90058F090004F740AF090003BE0900050F0D9
:103ED9007BFF7A0579CA1246471246727F0D121383
:103EE9000A900006E0FF1212DB900007E0FF1212B1
:0D3EF900DB7F1E12130A9000007432F022CD
:10262D0012349ED3900067E09400900066E0940011
:10263D00400A12464190000074FAF022900066E0C4
:10264D00FEA3E0FF90045075F009122C6AEE75F0B0
:10265D0009A42583F583E493900045F0900451750A
:10266D00F009EF122C6AEE75F009A42583F583E4C9
:10267D0093900046F0900066A3E090045275F00927
:10268D00122C6AEE75F009A42583F583E49390006E
:10269D0047F090045375F009EF122C6AEE75F009AE
:1026AD00A42583F583E493900048F0900066A3E0A1
:1026BD0090045475F009122C6AEE75F009A4258367
:1026CD00F583E493FD900049F090045575F009EF02
:1026DD00122C6AEE75F009A42583F583E49390001E
:1026ED004AF0900066A3E090045675F009122C6A2A
:1026FD00EE75F009A42583F583E49390004BF090DB
:10270D00045775F009EF122C6AEE75F009A42583B4
:10271D00F583E49390004CF0900066A3E09004588C
:10272D0075F009122C6AEE75F009A42583F583E482
:10273D009390004DF0ED6015900049E075F010A4F8
:10274D00244AF9740535F0FA7BFF12464790004A8A
:10275D00E0FF601175F010A4244AF9740535F0FA04
:0E276D007BFF124678900045E0900000F022BD
:104795003028079000007401F02290003C742EF040
:1047A50090003D7407F07BFF7A0579DA12464712CF
:0E47B50046727F1E12130A9000007432F0222A
:10439100302F07900000742FF02290000BE064385A
:1043A1006005A3E0B4390A12464190000074FAF0A6
:1043B100227BFF7A06798A12464790000BE0540F60
:0943C100F54B9000007430F0226D
:103FE50090000BE064386005A3E0B4390A1246413D
:103FF50090000074FAF0227BFF7A0579EA124647B1
:1040050090000BE0540FF54BD212D21A7535FF1202
:10401500187A7BFF7A0679BA124647C212C21A90FD
:06402500000074FEF02211
:103F9C0090000BE0540FF54B302602D21012188C07
:103FAC00302619203D04E53070F91218837BFF7A16
:103FBC000679BA12464790000074FEF0302719209B
:103FCC003B04E53070F91218837BFF7A0679BA123C
:093FDC00464790000074FEF0223B
:103B2300302956900001E0FF900035F0C2291212AF
:103B3300DB900035E0FF124C7A5021900035E0FF16
:103B430090003DE02404F582E43400F583EFF09027
:103B5300003DE004F0900000E004F022900035E026
:103B6300B42A079000007403F0227BFF7A06799A47
:0A3B730012464790000074FAF02299
:1036680030296A900001E0FF900035F0C22912125B
:10367800DB900035E0FFB42A0B90003CE09000009E
:10368800F0D22F22EFB4230B90003CE0900000F022
:10369800C22F22900035E0FF124C7A50219000355D
:1036A800E0FF90003DE02404F582E43400F583EF68
:1036B800F090003DE004F0900000E004F0227BFF71
:0E36C8007A06799A12464790000074FAF022B2
:10406F0030293F900001E0FF900035F01212DBC2C3
:10407F0029900035E0FFB42A0B90003CE09000003F
:10408F00F0D22F22EFB4230B90003CE0900000F011
:10409F00C22F227BFF7A06799A124647900000744E
:0340AF00FAF02202
:0A3D2F00900048E0FF7003302F38C9
:103D390012130A124A121230F28F6B900046E052A7
:103D49006BE56B60047F3180027F301212DB302F0C
:103D590017C22FE56B2430900024F09000347401D1
:083D6900F090000074F0F0225C
:0F3D710090004BE0FF12130A900000E004F022D4
:10402B00302940900001E0FF900035F0C2291212B8
:10403B00DB900035E0FFB42A079000007403F022F8
:10404B00124C7A500F900035E090000EF09000006B
:10405B00E004F0227BFF7A06799A12464790000023
:04406B0074FAF022D1
:10447100302932900001E0FF900035F0C229BF2AB7
:10448100079000007403F022900035E0B4230790F8
:104491000000E004F0227BFF7A06799A12464790E9
:0644A100000074FAF02295
:103B7D00124A1290006AEEF0A3EFF01230F28F6B42
:103B8D0090003E7401F090000EE0B43108900046B4
:103B9D00E0426B800E90000EE0B4301E900046E0C7
:103BAD00F4526B90006AE0FEA3E0FFAD6B1230B1F2
:103BBD00124C3290000074FEF0227BFF7A06799A47
:093BCD0012464790000074FAF062
:013BD60022CC
:10342900900048E0FF7003302F5612130A124A1217
:1034390090006AEEF0A3EFF0E4F56B900046E0FF30
:10344900E56BC39F502790006AE475F001122C5474
:10345900AFF0FE1230F28F6C7424256BF582E434E0
:1034690000F583E56CF01212DB056B80CE302F106E
:10347900C22FE56B04900034F090000074F0F02244
:1034890090003D740AF090004BE0FF12130A90007F
:0434990000E004F05B
:01349D00220C
:1033B000302975900001E0FF900035F0C22912120B
:1033C000DB900035E0FFB42A079000007403F02280
:1033D000EFB42308900000E004F08039124C7A50DA
:1033E00038900035E0FF90003DE0FE04F074042EBC
:1033F000F582E43400F583EFF0900046E02409FF05
:10340000E433FE90003DE0D39FEE6480F874809832
:103410004016900000E004F0227BFF7A06799A12B1
:09342000464790000074FAF02206
:10422F00302937900001E0FF900035F0C2291212BB
:10423F00DB900035E0FFB42A079000007403F022F2
:10424F00EFB42307900000E004F0227BFF7A067999
:0B425F009A12464790000074FAF0220B
:103C2F00124A1290006AEEF0A3EFF090003D740A72
:103C3F00F0E4F56B900046E0FFE56BC39F502790D3
:103C4F00006AE475F001122C54AFF0FE90003DE0D5
:103C5F00FD04F074042DF582E43400F583E0FD12C9
:103C6F0030B1056B80CE7BFF7A0679BA124647904A
:053C7F00000074FEF0DE
:013C8400221D
:1035F90030296B900001E0FF900035F0C2291212CA
:10360900DB900035E0FFB42A079000007403F02234
:10361900124C7A501A900035E0FF90003DE0FE040C
:10362900F074042EF582E43400F583EFF080107B0A
:10363900FF7A06799A12464790000074FAF02290B0
:103649000046E02409FFE433FE90003DE0D39FEEFD
:0F3659006480F87480984006900000E004F0222E
:102C9C00900048E0FF7006202F03022D4712130A04
:102CAC00124A1290006AEEF0A3EFF01230F21210FA
:102CBC00C5900046E0B40110900063E0FF1212DBF7
:102CCC00900063E0900024F0900046E0B402209065
:102CDC000062E0FF1212DB900063E0FF1212DB9047
:102CEC000062E0900024F0900063E0900025F090EA
:102CFC000046E064037030900061E0FF1212DB903C
:102D0C000062E0FF1212DB900063E0FF1212DB9016
:102D1C000061E0900024F0900062E0900025F090BB
:102D2C000063E0900026F0302F11C22F900046E097
:102D3C00900034F090000074F0F02290004BE0FF13
:102D4C0012130A90003D740AF0900000E004F02287
:103F060012111B5002803B1210F38F6B90004CE095
:103F1600FFE56BC39F402B90004DE0FFE56BD39F01
:103F26005020124A1290006AEEF0A3EFF0AD6B1229
:103F360030B17BFF7A0679BA12464790000074FECC
:0B3F4600F02212464190000074FAF0D7
:013F5100224D
:103D800012111B5002803F1210F38F6B90004CE019
:103D9000FFE56BC39F400B90004DE0FFE56BD39FA9
:103DA0004004E56B7020124A1290006AEEF0A3EF17
:103DB000F0AD6B1230B17BFF7A0679BA12464790AC
:0F3DC000000074FEF02212464190000074FAF0E9
:013DCF0022D1
:1031C000900048E0FF7003302F5E12130A124A127B
:1031D00090006AEEF0A3EFF01230F28F6B12313BE9
:1031E000E4F56B7461256BF582E43400F583E0FF50
:1031F0007424256BF582E43400F583EFF0746125C7
:103200006BF582E43400F583E0FF1212DB056BE519
:103210006BC3940440CD302F0FC22F900034740341
:10322000F090000074F0F02290004BE0FF12130ABF
:0C32300090003D740AF0900000E004F0F3
:01323C00226F
:104172007F0A1229FB8F6BE56B6012124A129000C4
:104182006AEEF0A3EFF0E56B14FD1230B1E56B7B44
:10419200FF600E7A0679BA12464790000074FEF06C
:0E41A200227A06793A12464790000074FAF02D
:0141B00022EC
:102E1C00900048E0FF7006202F03022EB712130A11
:102E2C00124A1290006AEEF0A3EFF01230F2121078
:102E3C00C590006AE475F001122C54AFF0FE12300C
:102E4C00F21210A9900062E0FF900024F0A3F0129F
:102E5C0012DB900063E0FF1212DB90006AE475F065
:102E6C0001122C54AFF0FE1230F21210A990006136
:102E7C00E0FF900026F0900062E0900027F09000B8
:102E8C0063E0900028F01212DB900062E0FF121257
:102E9C00DB900063E0FF1212DB302F0FC22F90008B
:102EAC00347405F090000074F0F02290004BE0FFB9
:102EBC0012130A90003D740AF0900000E004F02216
:102D5C0090000EE0540F75F00AA4FFA3E0540F2F5F
:102D6C00F56B900011E0540F75F00AA4FDACF090D7
:102D7C000010E0540F75F064A42DFFE5F03CFE90BC
:102D8C000012E0540F7C002FFFEC3EFEE56BC39469
:102D9C00014019E56BD394145012C3EF9401EE94D7
:102DAC00004009D3EF94FAEE9400400A1246419089
:102DBC00000074FAF022124A1290006AEEF0A3EFAF
:102DCC00F090006AE475F001122C54AFF0FEAD6B7C
:102DDC001230B1900011E0540F75F00AA4FF90006E
:102DEC0010E0540F75F064A42FFF900012E0540F04
:102DFC002FF56B90006AE0FEA3E0FFAD6B1230B1D3
:0F2E0C007BFF7A0679BA12464790000074FEF0F9
:012E1B002294
:101E4E007F0D1229FBEF701A900011E0B43010A331
:101E5E00E0B4300BA3E0B43006A3E06430600302BC
:101E6E001F47900015E0FF64306004EFB4350E900C
:101E7E000016E0540FD394054003021F479000153F
:101E8E00E0FF64316004EFB4361190001AE0B42024
:101E9E0007900019E0B42003021F47900015E0FFE1
:101EAE0064326004EFB43711900019E0B42007904B
:101EBE000018E0B42003021F47900015E0FF6433C2
:101ECE006004EFB43809900016E0B42002806A90E6
:101EDE000015E0FF64346005EF64397066900016FB
:101EEE00E0540F75F00AA4FFA3E0540F2FF56B908A
:101EFE000019E0540F75F00AA4FDACF0900018E044
:101F0E00540F75F064A42DFFE5F03CFE90001AE02E
:101F1E00540F7C002FFFEC3EFEE56BC3940140197D
:101F2E00E56BD394145012C3EF9401EE9400400964
:101F3E00D3EF94FAEE9400400A12464190000074DA
:101F4E00FAF022124A1290006AEEF0A3EFF090001F
:101F5E003D740AF0E4F56B900046E0FFE56BC39F1D
:101F6E00502790006AE475F001122C54AFF0FE90E9
:101F7E00003DE0FD04F074042DF582E43400F58399
:101F8E00E0FD1230B1056B80CE7BFF7A0679BA1276
:081F9E00464790000074FEF0BC
:011FA6002218
:10323D00900048E0FF7003302F5B12130A124A1200
:10324D0090006AEEF0A3EFF0E4F56B900046E0FF1E
:10325D00E56BC39F502C90006AE475F001122C545D
:10326D00AFF0FE1230F28F6C7424256BF582E434CE
:10327D0000F583E56CF07E001230F21212DB056B67
:10328D0080C9302F10C22FE56B04900034F09000F0
:10329D000074F0F02290004BE0FF12130A90003DF5
:0B32AD00740AF0D22C900000E004F046
:0132B80022F3
:10374300302965900001E0FF900035F0C229BF2ABF
:10375300079000007403F022900035E0FFB42308C3
:10376300900000E004F0803DEF547FFF1212DB90E5
:103773000035E0547FFF90003DE0FE04F074042E1A
:10378300F582E43400F583EFF0900046E02409FF6E
:10379300E433FE90003DE0D39FEE6480F87480989C
:0937A3004006900000E004F02251
:103DD00030294B900001E0FF900035F0C229BF2A46
:103DE000079000007403F022900035E0FFB4230B2D
:103DF000900000E004F0E004F08010124C7A500FC4
:103E0000900035E0900040F0900000E004F0227B4C
:0F3E1000FF7A06799A12464790000074FAF02262
:103014002029030230B0900001E0FF900035F0C297
:1030240029BF2A079000007403F022900035E0FFC6
:10303400B4230A900000E004F0E004F022124C7A79
:10304400505B900040E0540F75F00AA4FF900035E7
:10305400E0540F2FF0E09008B393FF900035F01286
:1030640012DB900035E0FF90003DE0FE04F07404B4
:103074002EF582E43400F583EFF0900046E0240955
:10308400FFE433FE90003DE0D39FEE6480F874804B
:1030940098900000E0400304F02214F0227BFF7AB1
:0D30A40006799A12464790000074FAF02257
:1049C400302609900080E0F565120FCF302803E40B
:1049D400F56530270B30240575650A800375652855
:0749E400900000E004F02246
:1037AC00E5657063122AE9900045E0122C7637DC4F
:1037BC006437E16E37E17837E18237E18C37E69692
:1037CC0037EBA037F0AA37F5B437FABE000037FD57
:1037DC00124B82801C1247058017124D1580121255
:1037EC004D16800D124D178008124D188003124D86
:1037FC001930260D90007FE0F55C900000E004F09D
:08380C00229000007401F0227B
:0E4C8900E55C7009120FD59000007401F02256
:103BD70030260D900080E0F565120FCFE56570FC8B
:103BE700302707756505E56570FCE4F56B30270C34
:103BF700124CD2121074124CF812107430260C1298
:103C07004CDD121074124CF8121074056BE56BC37F
:103C1700940540D930260A90007FE0F55CE55C709A
:073C2700FC9000007401F0A5
:013C2E002273
:014D1100227F
:014D1200227E
:014D1300227D
:1036D60030270A2024079000007401F02230260DBE
:1036E600900080E0F565120FCFE56570FC30270786
:1036F600756505E56570FC302615124CDDE4F56B45
:10370600121074056BE56BC3940A40F4124CF83042
:103716002715124CD2E4F56B121074056BE56BC3DA
:10372600940A40F4124CF830260A90007FE0F55CCB
:0C373600E55C70FC1243CAE4900000F057
:013742002264
:014D1400227C
:1041B100303D3B202938756664E540547FFF90020D
:1041C1006E93900001F0302C0EE54030E709EF903E
:1041D100027E93900001F0D229C23D900001E0B42B
:0F41E1002307900002E004F022E4900002F02295
:1041F000303B3B202938756664E53E547FFF9002D2
:104200006E93900001F0302C0EE53E30E709EF9000
:10421000027E93900001F0D229C23B900001E0B4ED
:0F4220002307900002E004F022E4900002F02255
:101A1400202A03021B81302903021B81900002E06B
:101A2400F56BE4F0756664124D0BD229BF30079054
:101A340000017430F022BF31079000017431F022AC
:101A4400BF32079000017432F022BF3307900001C7
:101A54007433F022BF34079000017434F022BF3590
:101A6400079000017435F022BF36079000017436E8
:101A7400F022BF37079000017437F022BF38079077
:101A840000017438F022BF39079000017439F02244
:101A9400BF23109000017423F0AF6B056B9000021C
:101AA400EFF022BF2A07900001742AF022BF4107F9
:101AB4009000017441F022BF42079000017442F08B
:101AC40022BF43079000017443F022BF64079000D3
:101AD400017444F022202C03C22922BF6107900024
:101AE400017461F022BF62079000017462F022BFAA
:101AF40063079000017463F022BF640790000174CF
:101B040064F022BF65079000017465F022BF660788
:101B14009000017466F022BF67079000017467F0BB
:101B240022BF68079000017468F022BF6907900023
:101B3400017469F022BF6A07900001746AF022BF41
:101B44006B07900001746BF022BF6C079000017466
:101B54006CF022BF6D07900001746DF022BF6E0718
:101B6400900001746EF022BF6F07900001746FF053
:0D1B740022BF70079000017470F022C2299A
:011B81002241
:0B4C97007F209000047420F0A3DFFCDD
:014CA20022EF
:0F4C7A00EFC394304007EFD39439500122C32287
:10349E0090000DE0FD6420602E90000CE0540F753E
:1034AE00F00AA4FBAAF090000BE0540F75F064A490
:1034BE002BFFE5F03AFEED540F7C002FFFEC3E9013
:1034CE000066F0A3EF803190000CE0FD64209000C8
:1034DE000B601AE0540F75F00AA4FFED540F7C0038
:1034EE002FFEEC35F0900066F0A3CE800BE0540F6B
:1034FE00FF900066E4F0A3EFF0E024FFF09000668A
:05350E00E034FFF02293
:1038140090000AE0FD6420602B900009E0540F75CD
:10382400F00AA4FBAAF0900008E0540F75F064A419
:103834002BFFE5F03AFEED540F7C002FFFEC3E9099
:103844000068802E900009E0FD6420900008601A52
:10385400E0540F75F00AA4FFED540F7C002FFEEC2A
:1038640035F0900068F0A3CEF022E0540FFF9000F2
:0738740068E4F0A3EFF0226D
:104A5700900006E0540F75F00AA4FFA3E0540F2F4F
:104A6700900036F0D394004006E09415500122C31D
:014A7700221C
:103AC600E4FFEF75F003A424CAF582E43406F58317
:103AD600E493FE900005E0FDEE6D703BEF75F0039C
:103AE600A424CBF582E43406F583E493FE90000625
:103AF600E0FDEEB50521EF75F003A424CCF582E4D4
:103B06003406F583E493FE900007E0FDEEB5050765
:0C3B1600900037EFF0D3220FBF33A7C39D
:013B22002280
:1039A700E4FF75F003EFA42463F582E5F03407F52F
:1039B70083E493FE900005E0FDEE6D703D75F00326
:1039C700EFA42464F582E5F03407F583E493FE90D1
:1039D7000006E0FDEEB5052275F003EFA42465F5BA
:1039E70082E5F03407F583E493FE900007E0FDEEEF
:0F39F700B50507900038EFF0D3220FBF70A4C3BF
:013A0600229D
:1029FB0074042FF582E43400F583E0FD64317069D3
:102A0B00FE74052FF582E43400F583E0FCEE75F0DF
:102A1B0003A424CAF582E43406F583E4936C704274
:102A2B0074062FF582E43400F583E0FCEE75F003B9
:102A3B00A424CBF582E43406F583E493B504237424
:102A4B00072FF582E43400F583E0FCEE75F003A468
:102A5B0024CCF582E43406F583E493B50404EE0448
:102A6B00FF220EBE339B7F0022ED6432706DFE742D
:102A7B00052FF582E43400F583E0FD75F003EEA439
:102A8B002463F582E5F03407F583E4936D704574A8
:102A9B00062FF582E43400F583E0FD75F003EEA418
:102AAB002464F582E5F03407F583E493B5052574CA
:102ABB00072FF582E43400F583E0FD75F003EEA4F7
:102ACB002465F582E5F03407F583E493B50505EE4F
:0D2ADB002434FF220EBE70977F00227F0082
:012AE80022CB
:10313B00EFC3943390006150397431F0EF75F003A5
:10314B00A424CAF582E43406F583E493900062F07C
:10315B00EF75F003A424CBF582E43406F583E493F6
:10316B00900063F0EF75F003A424CCF582E43406F1
:10317B00803A7432F075F003EFA424CAF582E5F0BF
:10318B003406F583E493900062F075F003EFA4240A
:10319B00CBF582E5F03406F583E493900063F0758C
:1031AB00F003EFA424CCF582E5F03406F583E49329
:0531BB00900064F02209
:104BF300900006E0540F75F00AA4FFA3E0540F2FB2
:054C0300900039F022D1
:104C0800900006E0540F75F00AA4FFA3E0540F2F9C
:054C180090003AF022BB
:104C1D00900006E0540F75F00AA4FFA3E0540F2F87
:054C2D0090003BF022A5
:064641007BFF7A06790AF6
:064647008B6C8A6D896E88
:10464D007F0112130AE4F56FAB6CAA6DA96E856F2D
:10465D0082758300122BD2FF1212DB056FE56FC33B
:04466D00941040E481
:014671002226
:064672007BFF7A06795A75
:064678008B6C8A6D896E57
:10467E007F1112130AE4F56FAB6CAA6DA96E856FEC
:10468E0082758300122BD2FF1212DB056FE56FC30A
:04469E00941040E450
:0146A20022F5
:104A1200900050E0FF90004FE08FF0A4FF90004E16
:104A2200E07C002FFFEC35F0FE900047E02FFFEC1A
:034A32003EFE2223
:104C3200900049E075F010A42452F9740A35F0FA94
:054C42007BFF02467833
:034D0B007F032201
:1049EB00E4F56BAF6B7E001230F2746C256BF582C5
:1049FB00E43400F583EFF0056BE56BC3942340E3E0
:064A0B0090006CE0F521B3
:014A11002282
:104B8200302608900024E0FF124CAF302708900036
:074B920024E0FF124CA322F6
:10470500E4F56B900034E0FFE56BC39F5021742402
:10471500256BF582E43400F583E0F56C302604FF63
:0F472500124CAF302705AF6C124CA3056B80D43C
:014734002262
:014D1500227B
:014D1600227A
:014D17002279
:014D18002278
:014D19002277
:0C4CA300124CE8121074124CFF02107446
:0C4CAF00124CF0121074124CFF02107432
:102AE900E4F56BF56CF56D900067E02401FF90004B
:102AF90066E03400FEC3EF940AEE94005005A3E0AB
:102B090004F56DD3EF9463EE9400404C900067E0B8
:102B19002401FB900066E03400FA7C007D64AF0379
:102B2900FE122BFF8F6BEF75F064A4FFC3EB9FFFC1
:102B3900EA95F0FE7C007D0A122BFF8F6CA3E0045E
:102B4900FFE56B75F064A4FEC3EF9EFFE56C75F0BD
:102B59000AA4FEC3EF9EF56D900067E02401FF9083
:102B69000066E03400FED3EF9409EE940040197C2E
:102B7900007D0A122BFF8F6CA3E004FFE56C75F052
:102B89000AA4FEC3EF9EF56D7430256BF56B7430A6
:102B9900256CF56C7430256DF56D302614AF6B120C
:102BA9004CAFAF6C124CAFAF6D124CAF7F2A124CC9
:102BB900AF302714AF6B124CA3AF6C124CA3AF6D9F
:082BC900124CA37F2A124CA359
:012BD10022E1
:103513002A2A3132333435362A2A2A2A31323334AD
:1035230035302A2A44313233343536373839302A64
:103533002341424320202056455253494F4E2031C8
:103543002E3420202020414C41524D2053595354B6
:10355300454D2020202041435449564520414C41AC
:10356300524D20202041435449564520524553543F
:103573004F52452020205452414E534D49545449F3
:043583004E4720206F
:102ECC00303025C230E540540F903527939000AC3C
:102EDC00F01238DF754D3290009EE004F03009148A
:102EEC001244DC1242A5800CE54D7008900099F05C
:102EFC009000A9F030313DC231E53E540F9035279A
:102F0C00939000ABF012387B754E3290009EE0042B
:102F1C00F0302403200806202406300A0312426AEB
:102F2C003024032008032024031244A72024111268
:102F3C004579800CE54E700890009AF09000A8F04E
:102F4C00302B19300B2212387B754F32124D0E90EC
:102F5C00009DEFF0C22B1242E0024511E54F7008C4
:092F6C0090009BF09000AAF022F5
:1044A70090009AE0FF04F0EF90351393FF9000AB74
:1044B700E0FEEF6E6011EEB42A0890009A7401F0E6
:1044C7008005E490009AF090009AE0B40A06E4F0C0
:0544D700D227D23222C1
:1044DC00900099E0FF04F0EF90351393FF9000AC3F
:1044EC00E0FEEF6E6011EEB42A089000997401F0B2
:1044FC008005E4900099F0900099E0B40A06E4F08D
:05450C00D226D232228C
:1045110090009BE0FF04F0EF90351393FF90009D16
:10452100E0FEEF6E6011EEB42A0890009B7401F07A
:104531008005E490009BF090009BE0B40A06E4F053
:05454100D228D2322255
:10426A009000A8E0FF04F0749F2FF582E43400F573
:10427A0083E0FF9000ABE0FEEF6E6011EEB423081E
:10428A009000A87401F08005E49000A8F09000A8BE
:0B429A00E0B40906E4F0D227D2252290
:1042A5009000A9E0FF04F0749F2FF582E43400F537
:1042B50083E0FF9000ACE0FEEF6E6011EEB42308E2
:1042C5009000A97401F08005E49000A9F09000A980
:0B42D500E0B40906E4F0D226D2252256
:1042E0009000AAE0FF04F0749F2FF582E43400F5FB
:1042F00083E0FF90009DE0FEEF6E6011EEB42308B6
:104300009000AA7401F08005E49000AAF09000AA41
:0B431000E0B40906E4F0D228D2252218
:1045790090009CE0FF04F0EF90351D93FF9000AB95
:10458900E0FEEF6E6011EEB42A0890009C7401F011
:104599008005E490009CF090009CE0B40A04E4F0EB
:0345A900D23322E8
:10481F0090009F7423F0A3F0E4FF746D2FF582E4F2
:10482F003400F583E0FE74A12FF582E43400F583A4
:0C483F00EEF00FBF06E49000A77423F019
:01484B00224A
:1043CA001212387BFF7A3579471246477BFF7A35D6
:1043DA0079371246787530147F10900051E4F0A3B3
:1043EA00DFFC7F10E53070FC1213241213337F01B7
:0843FA0012130AE490009EF08A
:014402002297
:10387B0090009EE0FED3940F50129000ABE0FF74CB
:10388B00512EF582E43400F583EF80437F01121350
:10389B000AE4F56B7452256BF582E43400F583E092
:1038AB00FF7451256BF582E43400F583EFF074510E
:1038BB00256BF582E43400F583E0FF1212DB056B18
:1038CB00E56BC3940F40CD9000ABE0FF900060F030
:0338DB001212DBEB
:0138DE0022C7
:1038DF0090009EE0FED3940F50129000ACE0FF7466
:1038EF00512EF582E43400F583EF80437F011213EC
:1038FF000AE4F56B7452256BF582E43400F583E02E
:10390F00FF7451256BF582E43400F583EFF07451A9
:10391F00256BF582E43400F583E0FF1212DB056BB3
:10392F00E56BC3940F40CD9000ACE0FF900060F0CA
:03393F001212DB86
:013942002262
:034D0E007F012200
:10187A00754A0012189550FB22754A0012191E501B
:10188A00FB22754A001218D550FB22758400E54ADE
:10189A0075F003A49018A27302193A0219490219A1
:1018AA006702195002197302197A02198202194938
:1018BA000219900219500219A00219A902193A0232
:1018CA0019490219B70219500219C3758400E54A69
:1018DA0075F003A49018E27302193A021949021921
:1018EA006702195002197302197A02193A02194940
:1018FA0002196702195002197302197A021973023E
:10190A00197A0219820219490219C50219500219D3
:10191A00A00219C3758400E54A75F003A490192B37
:10192A007302193A0219490219B70219500219C366
:10193A00C2FA1219D51219D5759B00054AC322306D
:10194A00F902054AC32230F912E59A20E7FB121977
:10195A00D5D2FA1219D51219D5054AC322C2FA12DA
:10196A0019D5759B04054AC322752F1E054AC32241
:10197A00E52F7002054AC322C2FA1219D51219F6C6
:10198A00F59B054AC322C2FA1219D5121A05440751
:10199A00F59B054AC3221219E7F530054AC3227599
:1019AA00840F30DE04E5307002054AC322C2FA12FF
:1019BA0019D5759B08054AC322D322C2FA1219D532
:0919CA00121A054405F59B054ABB
:1019D300C32200000000000000000000000000001F
:1019E300000000229019EEE54B93225A5A5A5A5A94
:1019F300FAFAFA9019FDE54B932200B45AE12D87C8
:101A03007ADB901A0CE54B93220000000000008063
:011A13008052
:1035870075840F1200A41249EB12481F1243CAE4B4
:103597009000B6F09000B3F09000AFF012431B120A
:1035A70043561232B9122ECC123943303305123337
:1035B70035C233303228C2327F0C121351124B4DB1
:1035C7001249EB12481FC226C227C228E4F56A1225
:1035D7001074056AE56AC3941E40F41243CA302585
:1035E700BB1245461249EB12481FC226C227C22802
:0235F70080AAA8
:10394300900041E07014121018400F120FE77569D0
:1039530064124CD2900041E004F0900041E0B401C5
:1039630010E569703E124CF875683C900041E00424
:10397300F0900041E06402701E12102A50051210EC
:10398300244007E568701020250D120FEF75696458
:10399300900041E004F022900041E0B40305E569A2
:0439A3007001F0229D
:10431B009000AFE0B40700503190432BF82828737E
:10432B0002434002434302434602434902434C02C9
:10433B00434F024352024AD7024C4702484C024BAE
:0B434B0099024BC7024AF61248782284
:104AD700900073E070059000AFF022C234C236E454
:0F4AE7009000B0F09000B1F09000AFE004F0222A
:104C4700124A78500C900088E0F55F9000AFE004BE
:024C5700F02249
:10484C00E55F701C900078E09000B0F0D234E490FA
:10485C0000B1F0900089E0F5609000AFE004F02228
:0C486C001247C340069000AFE014F02299
:104B99001247C35007900089E0F56022E56070066E
:074BA9009000AFE004F022D0
:104BC70090007AE09000B1F0E49000B0F0D2369017
:064BD70000AFE004F02233
:104AF600124A78500D900088E0F55F9000AFE00410
:0D4B0600F0229000B1E070049000AFF022AA
:10487800E55F701C900078E09000B0F0E49000B123
:10488800F0D234900089E0F5609000AF7403F02214
:0C4898001247C340069000AFE014F0226D
:104A7800300C0F90008AE0FFE532D39F4002D3222A
:104A8800C32290008AE0FFE532C39F500122C3226F
:1047C300300C1190008AE024F9FFE532D39F4002B8
:1047D300D322C32290008AE02407FFE433FEC3E51B
:0E47E300329FEE6480F8748098500122C32249
:104356009000B3E0B407005031904366F828287304
:1043660002437B02437E0243810243840243870267
:10437600438A02438D024B13024C590248D0024B2A
:0B438600B0024BDD024B301248A422B5
:104B1300900073E070059000B3F022C235C237E411
:0D4B23009000B4F0C2379000B3E004F0221F
:104C5900124A98500C90008BE0F55D9000B3E00487
:024C6900F02237
:1048D000E55D7019900079E09000B4F0D235E4F015
:1048E00090008CE0F55E9000B3E004F0221247F1F6
:0948F00040069000B3E014F02230
:104BB0001247F1500790008CE0F55E22E55E70062A
:074BC0009000B3E004F022B5
:104BDD0090007BE09000B5F0E49000B4F0D23790F7
:064BED0000B3E004F02219
:104B3000124A98500D90008BE0F55D9000B3E004B0
:0D4B4000F0229000B5E070049000B3F02268
:1048A400E55D701C900079E09000B4F0E49000B5F0
:1048B400F0D23590008CE0F55E9000B37403F022E2
:0C48C4001247F140069000B3E014F0220F
:104A9800300D0F90008DE0FFE533D39F4002D32205
:104AA800C32290008DE0FFE533C39F500122C3224B
:1047F100300D1190008DE024F9FFE533D39F400285
:10480100D322C32290008DE02407FFE433FEC3E5E9
:0E481100339FEE6480F8748098500122C32219
:103A0700202041435449564520414C41524D2020E6
:103A17002041435449564520524553544F5245205F
:103A270020205452414E534D495454494E4720206B
:103A3700202020202020202020202020202020207F
:103A47002020414C41524D2050414E454C202020D2
:103A5700202020202020202020202049444C4520C1
:1032B9009000B6E0122C7632FD0033000133030290
:1032C900331803330604330905330C0A33180B3357
:1032D9000F0C33120D331514331815331A16331D09
:1032E9001733201E33181F332620332921332C325C
:1032F9000000332F024B68022F750246A30245AC2A
:103309000248F90244030245DE0249220246D480FA
:103319000902473502494B02443A024CC702476544
:0C3329000249740228C6E49000B6F022AD
:104B6800900073E0FFB401079000B67401F022EFE3
:0A4B7800B402069000B67432F02279
:102F7500303425C234900078E09000B0F0E4900041
:102F8500B1F0D2387BFF7A3A79071246477BFF7A50
:102F95003A79371246788040303633C23690007A17
:102FA500E0FF602030381D9000B1F0E49000B0F0F3
:102FB5007BFF7A3A79171246477BFF7A3A793712BF
:102FC50046788025E49000B1F09000B0F022E561EC
:102FD500700D9000B0E060079000B6E004F022E5C7
:102FE50061700D9000B1E060079000B6740AF022A0
:102FF5009000B0E070189000B1E070127BFF7A3A53
:0F30050079471246477BFF7A3A7957124678226D
:1046A300300E09124D065004755B0522E55B702040
:1046B300F54A900074E0F54B90007EE0F55A120F36
:1046C300CF7BFF7A3A79271246789000B6E004F060
:0146D30022C4
:0B4CC700E55A70069000B6E004F022F1
:1045AC00D212D21A1218955028E4F54A9000B0E0B5
:1045BC00600214F0C23490007CE0F561E4F5629086
:1045CC00007DE0F56390007FE0F55C9000B6E004C0
:0245DC00F022CB
:1048F900C212C21AE55C7020120FD57BFF7A3A7991
:10490900371246789000B0E070097BFF7A3A793720
:09491900124647E49000B6F022BA
:10440300300E09124D065004755B0522E55B7026DC
:10441300F54A900076E0F54B90007EE0F55A120FD6
:10442300CF90007CE0F5617BFF7A3A7927124678DA
:074433009000B6E004F02246
:1045DE00D212D21A1218955028E4F54AC23690001B
:1045EE00B1E0600214F090007CE0F561E4F56290B9
:1045FE00007FE0F55C90007DE0F5639000B6E0048E
:02460E00F02298
:10492200C212C21AE55C7020120FD57BFF7A3A7967
:10493200371246789000B1E070097BFF7A3A7937F6
:09494200124647E49000B6F02291
:1046D400300E09124D065004755B0522E55B70200F
:1046E400F54A900075E0F54B90007EE0F55A120F04
:1046F400CF7BFF7A3A79271246789000B6E004F02F
:014704002292
:10473500D212D21A1218955026E4F54A9000B4E028
:10474500600214F090007CE0F562E4F56190007D74
:10475500E0F56390007FE0F55C9000B6E004F022A0
:10494B00C212C21AE55C7020120FD57BFF7A3A793E
:10495B00371246789000B4E070097BFF7A3A7937CA
:09496B00124647E49000B6F02268
:10443A00300E09124D065004755B0522E55B7026A5
:10444A00F54A900077E0F54B90007EE0F55A120F9E
:10445A00CF7BFF7A3A792712467890007CE0F562A2
:07446A009000B6E004F0220F
:10476500D212D21A1218955026E4F54A9000B5E0F7
:10477500600214F090007CE0F562E4F56190007F42
:10478500E0F55C90007DE0F5639000B6E004F02272
:10497400C212C21AE55C7020120FD57BFF7A3A7915
:10498400371246789000B5E070097BFF7A3A7937A0
:09499400124647E49000B6F0223F
:1028C600303426C234900078E09000B0F0E49000F6
:1028D600B1F0D2387BFF7A3A79071246477BFF7A06
:1028E6003A79371246780229C1303526C23590002A
:1028F60079E09000B4F0E49000B5F0D2397BFF7A2D
:102906003A79071246477BFF7A3A793712467802B8
:1029160029D2303636C23690007AE0FF6021303850
:102926001E9000B1F0E49000B0F07BFF7A3A791780
:102936001246477BFF7A3A79371246780229E3C274
:1029460036E49000B1F09000B0F022303735C2374F
:1029560090007BE0FF602030391D9000B5F0E490D8
:1029660000B4F07BFF7A3A79171246477BFF7A3A32
:1029760079371246788077C237E49000B5F0900038
:10298600B4F0229000B0E070249000B1E0701E9088
:1029960000B4E070189000B5E070127BFF7A3A79C7
:1029A600471246477BFF7A3A7957124678E56370B5
:1029B60043E561700D9000B0E060079000B67402C8
:1029C600F022E562700D9000B4E060079000B674E6
:1029D60014F022E561700D9000B1E060079000B63A
:1029E600740AF022E562700C9000B5E06006900073
:0529F600B6741EF02282
:054D0600120FFDB322B5
:1040F300191823A01296203D129623A01296276327
:104103001488203D148823A01488276316B8203D03
:1041130016B823A016B827631918203D191827636A
:1041230012962B8C14882B8C16B82B8C19182B8C6D
:0B4CD20075081575095ED23FD2132251
:0B4CDD0075081575095ED23FD21B223E
:074CF800C23FC213C21B22E0
:084CE800121CEDD240D214228F
:084CF000121CEDD240D21C227F
:091CED00E4F512F513F514F515E8
:101CF600EF122C761DF1231DE02A1D2E301D4031DA
:101D06001D52321D64331D76341D88351D9A361DCD
:101D1600AC371DBE381DCF391E02411E13421E248C
:101D2600431E354400001E4D9040F3E493F50D74B8
:101D36000193F50E9040F5021E449040F7E493F5AA
:101D46000D740193F50E9040F9021E449040FBE499
:101D560093F50D740193F50E9040FD021E449040DC
:101D6600FFE493F50D740193F50E904101021E44B4
:101D7600904103E493F50D740193F50E904105022D
:101D86001E44904107E493F50D740193F50E9041BE
:101D960009021E4490410BE493F50D740193F50E70
:101DA60090410D021E4490410FE493F50D7401938A
:101DB600F50E904111021E44904113E493F50D7403
:101DC6000193F50E9041158075904117E493F50D3A
:101DD600740193F50E904119806490411BE493F5CC
:101DE6000D740193F50E90411D805390411FE493AD
:101DF600F50D740193F50E9041218042904123E444
:101E060093F50D740193F50E90412580319041278D
:101E1600E493F50D740193F50E90412980209041CD
:101E26002BE493F50D740193F50E90412D800F90E0
:101E3600412FE493F50D740193F50E904131E4932F
:081E4600F50F740193F5102261
:074CFF00C240C21CC21422D6
:104A35003F313233343536010102030401010101EE
:104A450014050A6314FF320101FF323201018001AE
:024A55000180DE
:104B4D00E4F56BAF6B7E00E56B904A3593FD12304B
:0A4B5D00B1056BE56BC3942340E93A
:014B6700222B
:03000000024CBBF4
:0C4CBB00787FE4F6D8FD75819F023587F4
:102BD200BB010CE58229F582E5833AF583E02250B8
:102BE20006E92582F8E622BBFE06E92582F8E22202
:0D2BF200E58229F582E5833AF583E493221C
:102BFF00BC000BBE0029EF8DF084FFADF022E4CCBA
:102C0F00F875F008EF2FFFEE33FEEC33FCEE9DEC82
:102C1F00984005FCEE9DFE0FD5F0E9E4CEFD22EDC8
:102C2F00F8F5F0EE8420D21CFEADF075F008EF2F12
:102C3F00FFED33FD4007985006D5F0F222C398FD03
:052C4F000FD5F0EA22A0
:102C5400A3F8E0C5F025F0F0E58215827002158333
:062C6400E0C838F0E82290
:0C2C6A00A42582F582E5F03583F5832275
:102C7600D083D082F8E4937012740193700DA3A3ED
:102C860093F8740193F5828883E473740293686001
:062C9600EFA3A3A380DF01
:00000001FF
